:020000040000FA
:040000006622092843
:080008008D0A03198E0A0B1189
:10001000090064308C008D018E0196309E00FE2117
:10002000242258229E0B1028123091000D3090008F
:100030001D308F00C62119182A209918CC201919B3
:100040000F2199194821191AF020991AEA2124221E
:10005000582214288D214D2020306521023E1F3961
:100060009E008E0110088D0088001E0889006C21FA
:100070000F088C0088001E0A89006C211E08880069
:10008000203089006C21FE2124225822C6219908A3
:100090000319442899011A1408009C08031D5728C5
:1000A0000C088F000D0890000E0891000800013028
:1000B0001C06031D68280C088F000D0890000E0810
:1000C0009100E8308C0003308D008E0196200800EE
:1000D00002301C06031D7728A03092008630930062
:1000E000013094001F0A9E008620962008000330ED
:1000F0001C06031D8528403092007E309300053099
:1001000094001F0A9E008620962008008F0190010F
:10011000910112088F0713080318130F9007140892
:100120000318140F91079E0B8928080018309E00B1
:1001300011089700100896000F0895009101900192
:100140008F019401930192010310950D960D970D67
:10015000920D930D940D0E081402031DB5280D0881
:100160001302031DB5280C081202031CC6280C0834
:100170009202031C93031308FF3A031994030D081A
:100180009302031C94030E08940203148F0D900D28
:10019000910D9E0BA4280800203065219300643047
:1001A0009E0054225822C6219908031DD9289E0B6F
:1001B000D228130865218D00130A65218C008E0159
:1001C000FE2124225822C62199080319E128991CEE
:1001D000EE281308FE3E1F399300CF28990108002E
:1001E0009D08031DF9281A30910090001B308F00E4
:1001F000FE281930910090001C308F0024225822D4
:10020000C62199080319F028191E08299D09F0280C
:100210001D088800223089006C21990108009C0883
:10022000031D1929163091001530900005308F00FC
:10023000352901301C06031D242914309100143087
:10024000900005308F00352902301C06031D2F2930
:10025000173091001130900005308F00352917308C
:1002600091001130900018308F0024225822C621AE
:10027000990803190F29191D41291C0A03399C00EB
:100280000F29233089001C0888006C21990108007F
:100290000A301F02031C4E299F0148291F0A8C00A7
:1002A0008D01FE211B30910024225822C62199087D
:1002B00003194829991D5E299F0A4829243089007D
:1002C0001F0888006C219901080083128900831699
:1002D000081483120808080083168B01081555308E
:1002E0008900AA30890088148818742983120800AC
:1002F0009E0088011E0389006C219E0B792908004D
:1003000012308F00123090000E30910024225822BB
:10031000C62199080319802908009D080319952909
:100320008519C329051AC3299929851DC329051EC5
:10033000C32981018B0183168112811583124E22FC
:100340001330412205301B0685008B168B179D0844
:100350000319B6290230851DAB2981008D018E015C
:10036000051EB02901088B018C0008000230851998
:10037000B72981008D018E01051ABC2901088B0166
:100380008C00512208005122802108000130920087
:10039000FF3A8600FF3A5D22861FD8291207920095
:1003A0007F39031DC8299A019A099901542208002E
:1003B0009900920092091A08990512089A0054228D
:1003C0000800242258229A019A09C6219908031D7F
:1003D000E12908008F01910110309000013085194A
:1003E0008F00051A910024225822C6219908031D66
:1003F00008000130A607831CF329EA298F01900128
:1004000091018C080319172A8F0A0F080A3C031D53
:10041000152A8F01900A10080A3C031D152A900125
:10042000910A11080A3C03191E2A8C0B042A8D0814
:1004300003191D2A8D038C01042A080010308F0037
:1004400091000E309000080085010F084122013014
:100450001B0685004E225822512285011008412298
:1004600002301B0685004E225822512285011108B8
:10047000412204301B0685004E225822512254226C
:100480000800A5000030A50703300318013E8A00CC
:10049000250800237F3A1B0686000800F830650017
:1004A0000800FF30650008001B0885018601080070
:1004B000A4010000A40B592A08000000000000005D
:1004C0000000000000000000000008008B01512225
:1004D0008030660083168113831254223F306521D9
:1004E000C53A031D8922213065219B0022306521F8
:1004F0009D00233065219C00243065219F009A01D6
:100500009A09C621191889229918C1221919AC22F1
:1005100008004030782100308800213089006C21AB
:10052000FF308800223089006C210230880023309F
:1005300089006C2102308800243089006C21C5308C
:1005400088003F3089006C210C3091001B309000F6
:1005500012308F00E12108009A019A09C621191D65
:10056000BB2A7B308C008D01FE2124225822A60A52
:1005700003199B09AC2A213089001B0888006C21D3
:100580000800213078210C309100013090000630B5
:060590008F00E1210800CC
:1006000082073F3406345B344F3466346D347D34B6
:1006100007347F346F3477347C3439345E34793442
:100620007134403452345034093454341C3400345E
:100630003E34763408340134383431346E34AA34DC
:10064000AA34AA34AA34AA34AA34AA34AA34AA34BA
:10065000AA34AA34AA34AA34AA34AA34AA34AA34AA
:10066000AA34AA34AA34AA34AA34AA34AA34AA349A
:10067000AA34AA34AA34AA34AA34AA34AA34AA348A
:10068000AA34AA34AA34AA34AA34AA34AA34AA347A
:10069000AA34AA34AA34AA34AA34AA34AA34AA346A
:1006A000AA34AA34AA34AA34AA34AA34AA34AA345A
:1006B000AA34AA34AA34AA34AA34AA34AA34AA344A
:1006C000AA34AA34AA34AA34AA34AA34AA34AA343A
:1006D000AA34AA34AA34AA34AA34AA34AA34AA342A
:1006E000AA34AA34AA34AA34AA34AA34AA34AA341A
:1006F000AA34AA34AA34AA34AA34AA34AA34AA340A
:10070000AA34AA34AA34AA34AA34AA34AA34AA34F9
:10071000AA34AA34AA34AA34AA34AA34AA34AA34E9
:10072000AA34AA34AA34AA34AA34AA34AA34AA34D9
:10073000AA34AA34AA34AA34AA34AA34AA34AA34C9
:10074000AA34AA34AA34AA34AA34AA34AA34AA34B9
:10075000AA34AA34AA34AA34AA34AA34AA34AA34A9
:10076000AA34AA34AA34AA34AA34AA34AA34AA3499
:10077000AA34AA34AA34AA34AA34AA34AA34AA3489
:10078000AA34AA34AA34AA34AA34AA34AA34AA3479
:10079000AA34AA34AA34AA34AA34AA34AA34AA3469
:1007A000AA34AA34AA34AA34AA34AA34AA34AA3459
:1007B000AA34AA34AA34AA34AA34AA34AA34AA3449
:1007C000AA34AA34AA34AA34AA34AA34AA34AA3439
:1007D000AA34AA34AA34AA34AA34AA34AA34AA3429
:1007E000AA34AA34AA34AA34AA34AA34AA34AA3419
:1007F000AA34AA34AA34AA34AA34AA34AA34AA3409
:02400E00F93F78
:00000001FF
